:020000040800F2
:10500000381A0020D550000865820008757A00081B
:105010000000000000000000000000000000000090
:10502000000000000000000000000000558D000896
:105030000000000000000000E5880008558E000810
:10504000E7500008E7500008E7500008E750000864
:10505000E7500008295B0008E7500008E750000807
:1050600000000000E7500008515A0008E75000080F
:10507000E7500008E17E000800000000E75000084B
:1050800000000000E75000080000000000000000E1
:10509000E750000800000000E7500008E750000853
:1050A000E7500008E7500008E7500008CD950008D9
:1050B000E7500008E7500008000000000000000072
:1050C0000348854600F060FC00480047DDA3000867
:1050D000381A00200448804704480047FEE7FEE7EE
:1050E000FEE7FEE7FEE7FEE7F18E0008C15000088C
:1050F00030B50B46014600202022012409E00D4670
:10510000D5409D4205D31D469540491B25469540F7
:1051100040191546521E002DF1DC30BDF0B51FB40C
:105120000646002082B005464024019100901BE015
:10513000019922460F46304600F04EFB049A059B2B
:10514000801A994110D310461946224600F034FBCC
:10515000361A8F410197224601200021009F00F05E
:105160002BFB38184D4100902046641E0028DFDCE0
:10517000019B00982946324607B0F0BD03460B4319
:105180009B0703D009E008C9121F08C0042AFAD2FD
:1051900003E00B780370401C491C521EF9D2704783
:1051A000D2B201E00270401C491EFBD270470022BF
:1051B000F6E710B513460A4604461946FFF7F0FF16
:1051C000204610BD30B504460020034600E05B1CBD
:1051D000934203D2E05CCD5C401BF8D030BDF8B503
:1051E00002464A40D40F42004B0052085B089A42E4
:1051F00002D20246084611464A0023D0C30D4A0097
:10520000DDB2120EAD1A202D35DA49020126490A07
:10521000F6058A19002C00D0524220214F1B11465E
:10522000B9402A411018C20D9A4221D0002C17D043
:10523000012D08DCDA05801AD20F8019D207DBB203
:1052400000F0F6FAF8BDDA05801A012340001B06CB
:10525000C01880185A428018CA0F1043490007E04E
:105260004908C2071143DA05801A801940088018DE
:1052700000F0D6FAF8BD61000122511A001BF7E7D1
:105280000122D2075140AAE70122D2075040A6E7E7
:1052900070B502464A40D50F40004A00ED0740086D
:1052A0005208002814D0002A12D0C40DD30D410298
:1052B0000120C0055202490A520AE41A09181218BC
:1052C0007D34914201D3641C00E04900002C01DAD6
:1052D000002070BD0023914201D3891A0343400886
:1052E00049000028F7D100290AD0914202D10121BA
:1052F000C90705E0914201D2012101E00121C94322
:10530000E005C018401900F08BFA70BDF0B50746F3
:105310000846584087B0C00F049048000E46590018
:1053200040084908BC1A884105D2384631461E4615
:1053300017460B4602465800400810434CD0300D2B
:10534000039040055900400D490D0590401A029008
:10535000402872DA18030121000B09050843019067
:1053600004980092002805D00199524200208841FB
:1053700000920190029840210A1A0199009800F0C9
:105380001BFA05460C466B4607CB00F036FAC019EF
:105390007141039A0E0D0023D71756401A467A40E2
:1053A000164344D0049A002A2DD0029A012A039A67
:1053B00015DC1205C01A914101263605001C714109
:1053C000D20F059ED2070093019202962A462346E9
:1053D00000F074FA07B0F0BD38463146FAE716051A
:1053E000224A0F46B218C01AB74101210905001C14
:1053F0004F4100187F41114618187941E20F1043C0
:105400006D19644113E0E2076D0815436408C20793
:105410001443039A01261205C01A91413605001C57
:105420007141CE07400830434908C01851412A460F
:10543000234600F036FACDE7FFE70498012240004A
:10544000C117121A00238B4104983146C417381A29
:10545000A141EEE730B40124E407634030BC55E7D6
:1054600030B40124E407614030BC4FE70000E0FFA6
:10547000F0B51FB488B00B990998002448400999E9
:10548000C00F490049080991C0070B9900904900D5
:1054900049080B9109990898A64608431CD00B9916
:1054A0000A98084318D0099801244000420D48008A
:1054B000410D099824050003000B204309900B9827
:1054C0000003000B20430B9050181C494018002289
:1054D00001901446104605E0002001460DB0F0BDD5
:1054E000032801DA034600E003239C46C11A0AAEF2
:1054F0000AE05F0008ADED5B4F00F75B7D430027DE
:10550000AA187C41491C5B1E6145F2DD410004ABD9
:105510005A522104120C0A43240C401C0828DFDBD9
:10552000019802900099704601910090059B049AA1
:105530000799069800F0C2F9D0E700000DFCFFFFC4
:10554000F0B50C465C4085B0E40FE40703944C00D2
:1055500000266408590094464908024602962243F0
:1055600021D062460A431ED06200570D4A000E0346
:105570002303550D012402462C492405781B1B0BDF
:10558000360B401823432643614600901C46501AB0
:10559000B44103D30098401C009002E09218009898
:1055A0005B41002803DA0020014605B0F0BD002071
:1055B000012109050746864611E064461D46141B75
:1055C000B54106D36546521BB341744607430C43AD
:1055D000A646CD0740084908284392185B41054676
:1055E0000D43EAD11046184313D060461946504087
:1055F0007140084306D06046101AB34106D201221A
:10560000002306E000220123DB0702E00122D2434F
:105610005310009874460105381C6141029C039D9B
:105620000019694100F03DF9BFE70000FD030000EB
:10563000C217C10F504010B54018CA079623002169
:1056400000F0F6F810BD10B500229623114600F0C8
:10565000EFF810BD0EB5C217C10F5040CA07401871
:105660000021054B0293019200910A460B4600F07F
:1056700025F903B000BD0000330400000EB5054954
:105680000291002100910A460B46019100F016F9A3
:1056900003B000BD33040000410040020122400A73
:1056A000D205090E80187F2901DA0020704796295B
:1056B00003DC9622511AC8407047963988407047DB
:1056C00070B5CD0F4A0009030123090B1B051943CF
:1056D0000B4BED070024520D9A4201DA002070BDF9
:1056E000074B34339A4203DC9A1A00F075F802E053
:1056F0000449511888402C43F1D0404270BD00004D
:10570000FF030000CDFBFFFF4A0009030123090B43
:105710001B051943094B10B5520D9A4201DA0020BE
:1057200010BD064B34339A4203DC9A1A00F054F849
:1057300010BD03495118884010BD0000FF03000050
:10574000CDFBFFFFC20FD207400040080BD0C10DB8
:105750000723DB01C91840020905400A1143C208AA
:10576000400711437047002001467047CB0FDB070D
:10577000490010B5490802460A4307D00A0D07241C
:105780000903E401090B121B002A01DC002010BDF3
:10579000C900440F0C43C100E018D205801800F086
:1057A0003FF810BD0122D207002800DB101A0029A3
:1057B00000DB511A8142704710B5202A04DB0146F4
:1057C000203A9140002010BD914020239C1A0346AE
:1057D000E3401943904010BD10B5202A04DB084671
:1057E000203AD040002110BD0B46D340D0402024A9
:1057F000A21A91400843194610BD10B5202A06DBB5
:10580000CB170846203A1041C1170B4306E00B4660
:105810001341D0402024A21A91400843194610BDDC
:10582000002904DA401C490001D1400840007047BB
:1058300070B40024050C05D11024000402D1002905
:1058400021D01124050E01D100020834050F01D129
:105850000001241D850F01D18000A41C002801DB5C
:105860004000641C002908D020252E1B0D46F54061
:10587000A14000D001212943084301061B1B000A57
:10588000DB1D02D5002070BC7047DB05181880189E
:105890000029F8DA401C4900F5D170BC40084000EE
:1058A000704710B5002B08DA0024401C61419218A3
:1058B0005B411A4301D14008400010BDF0B51FB450
:1058C00082B005460C0003D0084603F03DFF02E01D
:1058D00003F03AFF20300246009021462846FFF7A9
:1058E0006BFF049B059A04460F4618431143084377
:1058F00014D0184610431BD0009840210A1A1846AD
:105900000599FFF769FF05460E46009A0599049828
:10591000FFF752FF084305D0012004E02046394636
:1059200007B0F0BD0020C11705430E432C43374399
:1059300000990E986305401A7905E40A00220C4389
:10594000FD0A0A3002D500200146E9E701051019D9
:1059500069410C9C0D9D00196941FFF7A2FFDFE72B
:1059600010B5002904DB0124E40740428C412146A4
:10597000002B04DB1C460123DB075242A341994262
:1059800000D1904210BD0000064C0125064E05E0F6
:10599000E36807CC2B430C3C98471034B442F7D350
:1059A000FFF792FB3CA700085CA7000838B5044647
:1059B000064805490068FFF79BFB604300E0401E76
:1059C00000900028FBD138BD40420F00EC000020C1
:1059D000F8B50446006881688907890F012902D15A
:1059E0000168C90722D18168114A1026114001259A
:1059F00000290ED18168294381600120FFF7D6FF7D
:105A000000F0A8FF07460CE000F0A4FFC01B0A2826
:105A100007D9606D30436065A06D2843A065012003
:105A2000F8BD20680068C043C007EDD10020F8BD74
:105A30001700008010B500231A4603E0845CE318C9
:105A40009BB2521C8A42F9D3D84380B210BD0000E9
:105A500010B5034800F03EFD024800F03BFD10BDCC
:105A6000D81500209015002030B5446C1C252C4022
:105A70000125A540046C6560046863608368102B91
:105A8000036803D099600068C26030BD9A60006806
:105A9000C16030BD1449012048720A4602205E32BE
:105AA000507203203C3A507204200E3A50720F4854
:105AB0000D4B0078087022310870203108770C49AE
:105AC0005A1C0878587149789971233318715971A3
:105AD000203318775977107551751A461E32107594
:105AE000517510765176704720110020BF000020BC
:105AF000D800002010B503F005F9202003F0A0F92C
:105B0000012004F0D1F9002003F09AF9044804F0D0
:105B10006FF8044804F012FB002004F047FB10BDAE
:105B2000A80000208380000070B505200121000737
:105B300000F000FF00240D4D002800D02C60022151
:105B40000B4800F0F7FE002808D10A482C600088B6
:105B50000A2148430849088003F04AFD012000F06B
:105B600021FE022000F01EFE70BD0000E4000020B7
:105B700000040050CC000020D60000207047000038
:105B800010B5084900224A6107494B684C15234368
:105B90004B604B68082423434B60C009C00102607E
:105BA00010BD000020160020002002407FB5002517
:105BB0000C460646039500F0C5FDE009029003A9D6
:105BC00001960095684600F055FD002804D000F0CD
:105BD0008DFD002004B070BD00F088FD0120F9E7C4
:105BE00010B5002302E0C45CCC545B1C9342FAD392
:105BF00010BD000010B5214A00219069C30520485E
:105C000004D54169022319434161911593699B05AC
:105C100005D5436901242343436163021943936912
:105C20005B0505D54369082423434361E301194318
:105C300093691B0505D5436904242343436163022B
:105C4000194393699B0405D5436910242343436199
:105C50006302194393699B0304D5446920231C43C1
:105C6000446119439369DB0305D543694024234309
:105C70004361A0020143916110BD00000020024079
:105C80002016002070B5054600F064FE0646184C4C
:105C90000AE0681C08D0002D04D000F05BFE801BD9
:105CA000A84201D9032070BDA069C007F1D1A06945
:105CB000800701D50220A061A069C00511D4A069A8
:105CC00080050ED4A06940050BD4A069000508D456
:105CD000A069800405D4A069800302D4A069C00330
:105CE00003D5FFF787FF012070BD002070BD0000C5
:105CF00000200240F8B51746002605460C4600F085
:105D000021FD09E029460220226800F0FDFC002860
:105D100004D1241D2D1D361DBE42F3D300F0E6FC38
:105D2000BE4201D20020F8BD0120F8BD10B50849DF
:105D300002460020054B497905E044001C5B944273
:105D400003D0401CC0B28842F7D310BD48120020D7
:105D50004800002010B500F0F2FD10BD10B5094854
:105D600000F09AFF80B2FFF789FC074A074BFFF764
:105D70007FFB0022064BFFF7E3FBFFF7C5FC80B279
:105D800010BD000088140020F853E3A59B843E401A
:105D900000408F40F8B53F493D488A7F0275C97F72
:105DA00041753D490A78027649784176384905209F
:105DB000133148720A2004F0B1F9002004F0C8F948
:105DC0003349002213310C2004F092FA00210C20F8
:105DD00004F0A0FA022004F0F1F9304D2D4C00211E
:105DE0000F2004F01BF92842E062F8D0E06A411C61
:105DF00040D02B4E2B4F40043ED58122D2010021B2
:105E00000F2004F04AFA0021102004F007F941069F
:105E10001F48490E0022633004F036F91C4D6335EB
:105E2000687A052825D102221B49681DFFF7CAF9A7
:105E300000281ED1A87A607116480422691C4030DF
:105E4000FFF79CF9206C00F033F8A08360792946B5
:105E500042000B3108465930FFF790F9124831885B
:105E60008088FFF745F938884143104801800220B7
:105E70002070F8BD02F01AFAA08B31880546FFF7B2
:105E800037F93888414309486D1E0180A583F8BD64
:105E90008111002048000020D800002000D02724D5
:105EA000C8000020C6000020200D0020C4000020F3
:105EB00010B504460E4800F0EFFE0E49C006C00EB5
:105EC000098805E02246C240D2070FD0401CC0B26C
:105ED0008842F7D3012005E02246C240D20705D010
:105EE000401CC0B28842F7D3491EC8B210BD0000A2
:105EF00088140020C800002010B5084800F096FA69
:105F00000A21064800F032FA044800F01DF9800525
:105F100003D5024800F01AF980B210BD2C140020FD
:105F2000F8B52F4D00220121284600F00CFDFFF7A7
:105F3000E3FFFFF788FB2B4E3146FFF7A9F92A4C08
:105F40000122A0601146284600F0FDFC2749A06808
:105F5000002588423EDB2078254F002815D025708B
:105F6000FFF7CAFFFFF76FFB3146FFF791F9A0601B
:105F7000FFF7E8FB00223B46FFF76CFA00221D4BBF
:105F8000FFF776FAFFF7F2FB6060A068FFF7DAFB35
:105F900000223B46FFF75EFA174A184BFFF768FAF4
:105FA00006460F466068FFF7CDFB134A144B52427A
:105FB000FFF75EFA32463B46FFF7A8F9FFF7D6FB3C
:105FC00010496060884201DD616004E0FF21C9057D
:105FD000C84200D365606068FFF75EFBC0B2F8BDE1
:105FE0000004005000401B442400002000006040DA
:105FF00000000C4000E064403333333333B33040AF
:10600000CCCCEC3F0000C842F8B50546044640350C
:10601000287C0026012808D0012028742068816887
:106020008907890F01290ED101E00220F8BD01681E
:10603000C90708D0606D2021084360650126002053
:1060400028743046F8BD616DFF220132914302226F
:1060500011436165C1688907890F0091C16889088A
:106060008900C1602068816892071143816000F057
:1060700071FC07460EE000F06DFCC01B0A2809D930
:10608000606D022188431021084360650020287458
:106090000120F8BD206880680028ECDB2068C1681A
:1060A000009A1143C160606D80088000401C6065EB
:1060B000C5E70000F8B506460D464036317C01299B
:1060C0000DD00121317401688A68520709D5416DEC
:1060D000202211434165002030740120F8BD0220C8
:1060E000F8BD174B6A68D80547109A42154C8A6A62
:1060F0002B6812D05B035B0B1A438A622968490341
:1061000005D5A1680143A1600A20FFF74FFC28686C
:10611000800312D5A06838430EE05B035B0B9A4303
:106120008A622968490302D5A1688143A160286871
:10613000800302D5A068B843A06000203074F8BD89
:106140000110000000270140406D70470068006C9E
:106150007047000070B5040006D0606D264600252B
:106160004036002802D006E0012070BDA5653574D8
:10617000204600F0D3F8606DC00603D4216888681B
:10618000400705D5606D1021084360653574EBE765
:10619000606DFF22013290430222104360658868DF
:1061A0008207920F5B48012A02D10A68D2072BD1DD
:1061B000032362689B079A4205D05B429A4202D051
:1061C0005B009A4209D10A69920092080A6121682B
:1061D0000A6963681A430A610CE00A69920092082E
:1061E0000A6181680F22920491438160816862682C
:1061F000114381602168CA6818239A43CA602168E4
:10620000CA68A3681A43CA60816801225206914392
:1062100081608168A28E5206114381602068816886
:10622000C90004D4816801221207114381602068EB
:10623000C168394A1140C1602069E168022825D04F
:1062400000200143204620300278037B52035B008C
:106250001A431143226B1143A26992031143E2696D
:10626000D20311432268D3681943D160616A0A4698
:10627000FF3AC23A05D0A26A11432268D368194393
:10628000D16042780121012A02D00BE00420D8E736
:106290000078002823D0606D202210436065A06D37
:1062A0000843A065E06B012820681FD00169C90779
:1062B00003D0016949084900016120684169C908A2
:1062C000C900416120684169A26B11434161A56524
:1062D000606D80088000401C6065002070BD2068F3
:1062E000C26801231B041A43C260DBE70269FF2373
:1062F0009B009A43026120680269236CA66C1A43D2
:10630000636C33431A430261206802690A430261E5
:10631000D3E70000002701401902FEFF10B586B048
:10632000044614216846FEF742FF0E492068884261
:1063300016D10D48416B421511434163C16A0122D8
:106340001143C162C06A6946104005900220009066
:1063500003200190002002900520000700F02EFA93
:1063600006B010BD0024014000100240F8B50446FC
:106370004069254640350E4608280BD02068C06885
:10638000C00709D0606D2021084360650020287493
:106390000120F8BD082700E00C2700F0DBFA009090
:1063A00011E0701C0FD0002E05D000F0D3FA009938
:1063B000401AB04207D9606D04210843606500208F
:1063C00028740320F8BD206800683842E9D0606D69
:1063D00001214902084360652068C16809058A0FE8
:1063E0000C21002A1BD12022125D002A17D102683D
:1063F000120714D5826853070122002B08DB43687B
:106400008B434360606D130298431043606506E060
:10641000606D202318436065A06D1043A065A069DE
:10642000002801D1206801600020F8BD70B5044645
:10643000216800208968490721D425464035297CF8
:1064400001291CD001212974E169012904D02046C9
:10645000FFF7BEFA002811D1616D0A4A1140FF22F0
:106460000132114361650021A165297422681C2154
:10647000116021688A6804231A438A6070BD022073
:1064800070BD0000FEF1FFFF70B500240146203111
:106490004A79022A03D00421C163012418E002686A
:1064A00013680E25AB431360026813685B085B003A
:1064B0001360436C1C221340012215469D40036C5F
:1064C0005D604A7100220A71816B002900D0884703
:1064D000204670BDF0B4016C0D6801680C68466C14
:1064E0001C2304221E401746B7402F420ED06707D8
:1064F0000CD50C68A40602D40C6894430C60416C63
:1065000019408A40016C4A60016B1AE00227B740CB
:1065100002462F402032002F17D0A70715D50C6850
:10652000A40605D40C680A25AC430C600121517106
:10653000446C02211C40036CA14059600021117180
:10654000C16A002918D0F0BC08470827B7402F427D
:1065500012D0240710D50C680E25AC430C60446C97
:1065600001211C400B46A340046C6360C163517160
:1065700000211171416BE4E7F0BC704770B5040075
:106580003CD01F48256814212818FEF7B1FD800073
:1065900060641C482064022120462030024641717C
:1065A00029681948E3680140A068666918432369AF
:1065B00033431843A3691843E3691843236A184314
:1065C000084328600121A0688903884210D00D4843
:1065D0008030836A656C1C210D400F26AE40B343AA
:1065E0008362656C63680D40816AAB400B438362D4
:1065F0000020E06301215171107170BD012070BD58
:10660000F8FFFDBF000002400F80FFFFF8B5044611
:106610008C46203001790025012909D00126067118
:1066200041790027012905D0077102252846F8BDC8
:106630000220F8BD02214171E76320680168490822
:106640004900016061462046FFF70EFA206B0028E2
:106650002068016801D00E2205E004229143016008
:10666000206801680A2211430160206801683143F3
:106670000160DBE7F8B51A4E0546307C0F4601286D
:1066800007D0012030741748FFF7FCFA010002D050
:1066900021E00220F8BD0020C04338606C6814E09F
:1066A0002046FFF76DFA0F48FFF7ECFA01460E4857
:1066B000426808239A434260426843159A43426005
:1066C000002901D03C6006E08034A8686A68C001F7
:1066D0008018A042E4D8002030740846F8BD0000BD
:1066E0002016002050C300000020024005484168E9
:1066F00002221143416041680122114341600020A0
:106700007047000000200240F8B50C4C1646207C73
:106710000F46012808D0012020740948FFF7B2FA7B
:106720000025002802D006E00220F8BD65613E6029
:106730000348FFF7A7FA2574F8BD000020160020D3
:1067400050C3000011484168C9070BD0EFF3108116
:1067500072B60F4AC2600F4AC26081F31088416866
:10676000C9070ED1416889070DD5EFF3108172B6C4
:10677000094A0261094A026181F310884068800772
:1067800001D5012070470020704700000020024022
:10679000EFCDAB8905040302BFAE9D8C1615141313
:1067A0007047000010B504494A69024202D04861AE
:1067B000FFF7F6FF10BD000000040140F8B500230C
:1067C0000124A2E027469F403A4070D04D68022D38
:1067D00001D0122D14D1DD08AD002D1800952D6AC1
:1067E0005E07AC46F50E0F26AE46AE406546B54395
:1067F000AC460E697546AE4065462E43009D2E623E
:106800004D68012D05D0022D03D0112D01D0122D80
:1068100016D185680326AC465D00AE46AE4065469F
:10682000B543AC46CE687546AE4065462E4386609D
:1068300046680D79BE43ED06ED0F9D40354345603A
:1068400006685F000325BD40AE46AE430D79B446F1
:10685000AE07B60FBE4065462E430660C668754655
:10686000AE438D68BD403543C5604D68ED004BD5E6
:10687000294D6E6B26436E639E08284DB600751930
:10688000AC46AD689E07360F0F27B740BD430527BE
:106890003F07B84201D1002715E0214FB84201D18E
:1068A000012710E01F4FB84202D102270BE02BE076
:1068B0001D4FB84201D1032705E01C4FB84201D15A
:1068C000052700E00627B7402F436546AF60184D07
:1068D0002E684F689643FF0300D516432E606E68FE
:1068E0004F689643BF0300D516436E60AE684F688D
:1068F0009643FF0200D51643AE60EE684F6896439C
:10690000BF0200D51643EE605B1C0A681546DD40E9
:1069100000D057E7F8BD0000001002400000014021
:106920000004005000080050000C0050001C0050F3
:10693000000401400069084000D00120704742690E
:106940004A4042617047002A01D0816170478162EC
:10695000704700000148006870470000E800002010
:1069600002480168491C016070470000E8000020EF
:1069700010B50848002401684022114301602046F8
:1069800000F00AF8002801D0012401E000F0B0F97D
:10699000204610BD0020024070B5054609487D2103
:1069A0000024C9000068FEF7A3FB00F045FE0028A4
:1069B00001D0012404E000222946501E00F0B8F95D
:1069C000204670BDEC00002070477047F8B52C4C95
:1069D0000126A078401CA0702671208B401C2083CB
:1069E000208902F0F5F9274DE888FEF72CFE2649AC
:1069F000FEF74EFC254F3968FEF7F1FB38600221A7
:106A00002348FFF797FF0027002809D027621F4877
:106A1000204A016820480091914212DD067011E081
:106A2000E888FEF710FE1849FEF732FC216AFEF7EF
:106A3000D6FB1A4920628842E9DB1A491848C86027
:106A4000E5E70770688F401EFEF7F2FD0099FEF73C
:106A5000A9FE05D86079002802D01348067001E02D
:106A600011480770688FFEF7EEFD08490968FEF7C8
:106A700099FE04D26079002801D003F033FDF8BDFF
:106A8000BC000020200D002000007A44E40000201B
:106A900000040050000040404E0000200000A040D4
:106AA0000400FA0500ED00E05C000020704770B5BE
:106AB00005000DD002202C462034A073284601F09A
:106AC00017FA284600F0BEF80020A073607370BD6E
:106AD000012070BD7047704710B50446006801681A
:106AE000C943C90708D18168C943C90704D1012135
:106AF00041602046FFF76AFF20680168C9438907A3
:106B000008D48168C943890704D402214160204622
:106B1000FFF75AFF20680168C943490708D4816814
:106B2000C943490704D404214160204600F0DEF83F
:106B300020680168C943090708D48168C943090767
:106B400004D4082141602046FFF7B0FF20680168A7
:106B5000C943C90608D48168C943C90604D41021B1
:106B600041602046FFF731FF20680168C94389066C
:106B700008D48168C943890604D420214160204695
:106B8000FFF7A9FF20680168C943490608D4816856
:106B9000C943490604D4402141602046FFF79AFFCB
:106BA00010BD0000F8B5040005D025462035A87BAF
:106BB000002802D006E00120F8BD002068732046BE
:106BC00000F052F80220A8732068C2688446636807
:106BD000012B04D00120A16AC005814201D11E20F1
:106BE000824315486169814201D01448024014482B
:106BF000A668024018463043676A266A3E4330431F
:106C0000A66A30431043012B03D00122D2059642DD
:106C100003D12369E2681A431043074A914205D021
:106C2000A2691143E2690243084610436146C86005
:106C30000120A8730020F8BDFFFF00003F1FFFFFE9
:106C4000F8F119FF10B500680549884207D10548D9
:106C5000816B4900490881630D2000F055F810BD93
:106C6000007C00400010024010B5006808498842CE
:106C70000CD10848816BC2041143816300220121B9
:106C80000D2000F055F80D2000F048F810BD000070
:106C9000007C0040001002400068C069704700009E
:106CA00070B50224034620339C730F4C2568E6041C
:106CB000354325600468E568B6123543E56005682C
:106CC000AE6801242643AE6005682E6926432E6116
:106CD0000568A96101684A610068016904221143DD
:106CE00001619C73002070BD0004014070470000EA
:106CF0000448416B012211434163816B020411433B
:106D00008163704700100240C106C90E012088400F
:106D1000014908607047000080E100E0C106C90E2B
:106D200001208840014908607047000000E100E050
:106D300010B501F099FA10BD02494A6882434A60D1
:106D4000704700000070004002480168821511433E
:106D5000016070470070004002494A6802434A607F
:106D6000704700000070004005480168022211438E
:106D700001600448016904221143016130BF70477A
:106D80000070004000ED00E00A4B1A689208920083
:106D900002431A600848036904221343036101296E
:106DA00006D040BF20BF20BF0169914301617047F9
:106DB00030BFF9E70070004000ED00E0F8B5044690
:106DC0000078544D800672D5524E0027403EB06B7D
:106DD000C00004D4B06BA9050843B06301274E4836
:106DE0000168C90511D40168821511430160FFF7DC
:106DF000B1FD009005E0FFF7ADFD0099401A642851
:106E000037D845480068C005F5D532680321090523
:106E100060680A400140914208D08103890F03292C
:106E200004D13168890301D50120F8BD2A69032105
:106E300009040A4022D0084090421FD020788006E2
:106E40001CD528692A6988430121C9040A432A619B
:106E50002A698A432A612861C0050FD5FFF77AFDA8
:106E6000009008E0FFF776FD0099411A2B48814217
:106E700001D90320F8BD28698005F3D5616888032E
:106E8000800F032805D132680005824301400A4380
:106E900032602869032261681204114008432861A6
:106EA000002F04D0B16B012000078143B16320782B
:106EB000C00705D0E868A168800880000843E86042
:106EC0002078800705D5E8680C218843E1680843ED
:106ED000E8602078400706D5E868032189028843E6
:106EE00021690843E8602078000706D5E868032197
:106EF0000903884361690843E8602078000606D5E5
:106F0000E868032189048843A1690843E8600020F8
:106F1000F8BD0000401002400070004088130000DF
:106F2000F8B50E4605007DD053480068C007C00F75
:106F3000B0420AD250480168490849003143016013
:106F40000068C007C00FB04271D128784B4C800751
:106F500005D5E068F0218843A9680843E0602878F7
:106F6000C00752D06868022817D0032818D02168BB
:106F7000012818D08905002959DAE16889088900B3
:106F80000143E160FFF7E6FC69680746022912D079
:106F900003291CD0012926D033E021688903EAE7C0
:106FA00021688901E7E74907E5E7FFF7D3FCC11B43
:106FB0003348814223D8E0680007800F0228F4D1CB
:106FC00023E0FFF7C7FCC11B2D48814217D8E068BA
:106FD0000007800F0328F4D117E0FFF7BBFCC11BAB
:106FE000274881420BD8E0680007800F0128F4D1C0
:106FF0000BE0FFF7AFFCC11B2148814201D9032000
:10700000F8BDE0680007800FF3D11B480168C9078D
:10701000C90FB1420DD901684908490031430160E7
:10702000006800E003E0C007C00FB04201D00120BB
:10703000F8BD2878400706D5E06807210902884393
:10704000E9680843E0602878000707D5E068072171
:10705000C90288432969C9000843E06000F036F896
:10706000E168084A0906090F515CC84006490860F2
:107070000020FFF791FCF8BD002002400010024004
:10708000881300001AA70008EC00002004480549F6
:107090000068C968044A4905490F515CC8407047F7
:1070A000EC0000200010024033A700080448054906
:1070B0000068C968044A8904490F515CC840704798
:1070C000EC0000200010024033A7000810B5184A59
:1070D000D1680C20084004280BD0082810D00C28B8
:1070E00010D050680004410F0120C003491C8840A3
:1070F00010BD1068C00601D50E4810BD0E4810BD69
:107100000E4810BD88020E4B000F185C0902D368B0
:10711000890F491CDB0301D5084A05E01268D20635
:1071200001D5044A00E0044A5043FDF7E1FF10BDD9
:107130000010024000093D000024F40000127A0013
:107140002AA70008FEB505007ED0FE4CE7680C209B
:10715000E66807400120000406402878C00747D0B1
:10716000082F05D00C2F0AD101200004864206D139
:10717000206880033CD568680028E5D038E001200D
:1071800069680004814203D121680143216011E054
:10719000052301221B0492049942216802D1114364
:1071A0002160F1E78143216021680140009120685E
:1071B00090432060686800280DD0FFF7CBFB00905B
:1071C00005E0FFF7C7FB0099401A64287AD82068C9
:1071D0008003F6D50CE0FFF7BDFB009005E0FFF75C
:1071E000B9FB0099401A6428F0D820688003F6D4CF
:1071F0002878800755D50923E868042F0DD00C2F77
:1072000001D1002E09D000283BD0216899430143C9
:107210002160FFF79FFB064627E02168490701D55B
:10722000002891D061681F22120291432A6912023C
:10723000114361602168994301432160FFF746FFD4
:10724000E16809060A0F00E079E1BF49895CC8409E
:10725000BE4908600020FFF79FFB002872D120E0A4
:10726000FFF778FB801B0228B0D820684007F7D5CD
:1072700060681F2109028843296909020843606088
:107280000FE02068400840002060FFF763FB0646DF
:1072900004E0FFF75FFB801B022897D820684007B7
:1072A000F7D42878C0065FD5002F0CD0A869002835
:1072B00049D02068FF21013108432060FFF74AFBD5
:1072C00006462DE0C0E02068800502D5A8690028A8
:1072D000A7D06068072149038843296A0843606092
:1072E0006068297F0002000A090608436060286A76
:1072F000410B0120C003491C8840E16809060A0FC0
:107300009149895CC840914908600020FFF744FB1F
:10731000002817D128E0FFF71DFB801B0228A3D807
:1073200020688005F7D56068072149038843296AEA
:10733000084360606068297F0002000A090608436C
:10734000606011E0E1E02168FF20013081432160AD
:10735000FFF700FB064604E0FFF7FCFA801B02285B
:1073600072D820688005F7D42878794E000724D594
:1073700068690028306910D0012108433061FFF7A7
:10738000E9FA009005E0FFF7E5FA0099401A0228B3
:107390005AD830698007F6D50FE0400840003061C8
:1073A000FFF7D8FA009005E0FFF7D4FA0099401AE9
:1073B000022849D830698007F6D42878400765D577
:1073C00000200290A06BC00006D4A06B0121090729
:1073D0000843A063012002905E480168C90511D4EA
:1073E0000168821511430160FFF7B4FA009005E0CF
:1073F000FFF7B0FA0099401A642825D8554800686C
:10740000C005F5D5FF20AA680130824203D1316959
:107410000143316111E001218902002A07D00523CF
:107420001B029A4203D132690A433261EFE73269A3
:1074300082433261306988433061A86800280FD0E8
:10744000FFF788FA009007E05EE0FFF783FA009903
:10745000411A4148814257D830698005F5D50DE081
:10746000FFF778FA009006E0FFF774FA0099411AE6
:107470003948814248D830698005F5D402980028FF
:1074800004D0A06B012109078843A063686A002823
:1074900064D00C2F3ED0012636060228206805D085
:1074A000B0432060FFF756FA05462FE0B043206056
:1074B000FFF750FA074604E0FFF74CFAC01B02281A
:1074C00022D820688001F7D4E96AA86AE2680843F4
:1074D000296BFD231B049A4311430843E060206895
:1074E00030432060FFF736FA054604E0FFF732FA32
:1074F000401B022808D820688001F7D52EE0FFF74E
:1075000029FA401B022801D90320FEBD2068800112
:10751000F5D423E00128F8D0E06801210904AA6A23
:10752000014091420BD10F218904EA6A0140914246
:1075300005D1032189050840296B88420ED001201E
:10754000FEBD0000001002401AA70008EC00002059
:107550004010024000700040881300000020EFE758
:1075600070B5040007D0002625464035A662687C29
:10757000002802D005E0012070BD2E74204600F0E6
:107580002FF802206874206801684022914301604E
:10759000A168606822690843E16811430843616992
:1075A00001220843A169520211400843E1690843DE
:1075B000216A0843A16A084321680860A069042180
:1075C000000C0840616A0843216848602068C1696E
:1075D00092009143C161666501206874002070BD0E
:1075E00010B586B0044614216846FDF7E0FD104949
:1075F0002068884219D10F48416B821411434163BE
:10760000C16A01221143C162C06A00211040059085
:10761000E020009002200190032003900291049149
:10762000052069460007FFF7C9F806B010BD000045
:107630000030014000100240094910B5401E884248
:1076400001D9012010BD074C60610321081F00F023
:107650000BFE0020A06107202061002010BD00006B
:10766000FFFFFF0000E000E070477047F8B50268D8
:107670000446D0691168936805072D0F5BD0DD07BC
:10768000ED0FFF2621360E402E4367D0C60706D0E9
:10769000CE0504D501261662E26F3243E267870702
:1076A00002220426002F06DADF0704D027683A6298
:1076B000E76F3743E767470706D5DB0704D0236842
:1076C0001E62E36F1343E367020709D520220A40D5
:1076D0002A4305D0236808221A62E36F1343E36745
:1076E000E26F002A2FD0800606D5880604D5216EC9
:1076F000002901D020468847E06F21688968490643
:1077000001D4000724D5204601F0D0FD206881680F
:10771000490619D58168402291438160E06E0028B6
:1077200012D020498163E06EFEF7AEFE00280AD039
:10773000E06E816B06E0850610D58D060ED5216EB4
:107740001CE020468847F8BD2046FFF78EFFF8BDB5
:107750002046FFF78AFF0020E067F8BDC50208D584
:107760005B0206D50120000510622046FFF77CFF72
:10777000F8BD030605D50B0603D5616E0029E0D1DF
:10778000F8BD4006FCD54806FAD5136820464021CE
:107790008B431360202161670021616600F069F965
:1077A000F8BD00000992000810B5040003D0606F16
:1077B000002802D007E0012010BD002170200155F3
:1077C000204600F027F824206067206801684908F7
:1077D00049000160204601F0B3FD0128ECD0606A49
:1077E000002802D0204601F0F1FB20684168092200
:1077F000D20291434160206881682A2291438160CE
:1078000020680168012211430160204601F044FC18
:1078100010BD0000F0B587B0064614216846FDF79C
:10782000C6FC2C493068884251D12B48416B01225B
:10783000920311434163C16A01221143C162C06ACC
:1078400000251040059003204002009002200327ED
:1078500001A9A1C104200490052069460007FEF794
:10786000ADFF1F4C1D48A560E56081C48027E56021
:10787000A7602020256160610002A0611848083CD3
:10788000FEF77CFE002801D0FEF778F9F466A662C8
:10789000144C1248214614382060032060601020E8
:1078A0000831A1C16561A561E56120462562FEF749
:1078B00065FE002801D0FEF761F9B46600220121BF
:1078C0001B20A662FFF734FA1B20FFF727FA07B048
:1078D000F0BD0000003801400010024030000240BE
:1078E00090150020D8150020F8B50446806F202898
:1078F0004DD100290BD0002A09D00123A0681B0319
:10790000984206D12069002803D1C80701D0012080
:10791000F8BD25466035287C012838D00120287420
:107920005820616502530026E6672220A067E06EBA
:10793000002819D01749C162E16E17480863E16E4B
:1079400016484863E06E13468663676D21683A46C1
:107950002431E06EFEF75AFE002805D01020E067C3
:107960002E7420206067D2E72E7420680168FF2201
:107970000132114301602068816801221143816056
:10798000206881684022114381600020F8BD0220F8
:10799000F8BD000065920008A39200081D9200083F
:1079A00070477047FFB50446406F83B017460D46D9
:1079B00020285CD1002D0AD0002F08D0A168C0017A
:1079C000814207D12069002804D1E80702D00120B4
:1079D00007B0F0BD204660300290007C012846D000
:1079E0000298012101740020E06721206067FEF702
:1079F000B1FF264640360190378277820120A16888
:107A00000003814202D12069002802D02F460025C0
:107A100011E000270FE000228021204601F0A4FDA4
:107A2000002815D1002F15D02168387888627F1C76
:107A3000708A401E7082708A019B00280698009010
:107A4000E9D100224021204601F08EFD002808D017
:107A50000320BDE728882168C005C00D8862AD1CE1
:107A6000E6E720206067029900200874B0E7022052
:107A7000AEE7704701490248C160FDE70400FA051E
:107A800000ED00E010B50524240700220421204663
:107A9000FEF759FF002208212046FEF754FF0A2076
:107AA00002F05FF8012204212046FEF74CFF0A2075
:107AB00002F057F8002204212046FEF744FF10BDD3
:107AC00010B505242407002204212046FEF73BFFC1
:107AD000012208212046FEF736FF0A2002F041F875
:107AE000012204212046FEF72EFF0A2002F039F879
:107AF000002204212046FEF726FF10BDF8B5002421
:107B00000526074625463607002204213046FEF7A3
:107B10001AFF0A2002F025F8012204213046FEF760
:107B200012FF6006040E08213046FEF703FF00280E
:107B300001D0641CE4B2052002F013F86D1CEDB214
:107B4000082DE1D3002F03D0FFF79CFF2046F8BD9E
:107B5000FFF7B6FFFAE770B505260546360700229F
:107B600004213046FEF7EFFE0024E80901D001228F
:107B700000E0002208213046FEF7E5FE6806050E0B
:107B80000A2001F0EEFF012204213046FEF7DBFE61
:107B90000A2001F0E6FF002204213046FEF7D3FE62
:107BA0000A2001F0DEFF641CE4B2082CDDD370BDB6
:107BB00010B505242407012208212046FEF7C3FE44
:107BC000012204212046FEF7BEFE002208212046A5
:107BD000FEF7B9FE0A2001F0C4FF0022042120466E
:107BE000FEF7B1FE10BD10B50524240700220421C4
:107BF0002046FEF7A8FE002208212046FEF7A3FE3D
:107C00000A2001F0AEFF012204212046FEF79BFE70
:107C1000012208212046FEF796FE0A2001F0A1FF6E
:107C200010BD70B505252D07002401220821284626
:107C3000FEF789FE062001F094FF01220421284668
:107C4000FEF781FE062001F08CFF07E0641CE4B221
:107C5000FA2C03D9FFF7C7FF012070BD0821284681
:107C6000FEF768FE0028F1D1002204212846FEF725
:107C70006AFE002070BD0000F8B501F03DFA01F089
:107C800077FA4C480068C0694B4E4C4F800700D5CE
:107C9000FE60FEF763F84A4C0246608849490028B6
:107CA00003D0401E608001200870087801218902FD
:107CB000454D00281CD0012804D0022804D00328F8
:107CC00006D115E0212A13D200222846FEF73BFEFA
:107CD0000121C9023C48FEF72DFE3C490025002841
:107CE00028D03B4805600846C079002802D006E04D
:107CF0000122EAE735490120C87101F079FC3348D7
:107D00000078632806D9002208212F48FEF71BFEC1
:107D1000012205E0012208212B48FEF714FE002273
:107D200001210520C9030007FEF70DFEA08C0128E4
:107D300003D01CE0CD710022EDE72648694608809B
:107D400072B680212448FDF731FF002804D00222BA
:107D500069462148FDF7CEFF62B620A001F0E4FCA1
:107D6000A58402F05BFC642001F0F4FEFE60608CF0
:107D7000012809D1124865844038058002F04EFC84
:107D8000642001F0E7FEFE60208C012806D12584E6
:107D900002F044FC642001F0DDFEFE600848134A56
:107DA00040380188914202D1C088002800D1FE608D
:107DB000F8BD0000101500200400FA0500ED00E0F9
:107DC000600D00205A00002000040050BC0000207C
:107DD000E4000020AAAA0000384A0008BDF8C8EB59
:107DE000C9FDBCB6C4A3CABD0D0A0000AA55000057
:107DF00008B53721202000F06EF80321212000F083
:107E00006AF84021222000F066F80821232000F0C3
:107E100062F8AA21302000F05EF80A4802210187AA
:107E2000322000F058F80121332000F054F85F218F
:107E3000202000F050F8684600F006F80A2001F013
:107E400090FE08BD200D002010B501460F2000F067
:107E500021F8002800D0012010BD10B50446FFF71E
:107E6000A7FE3220FFF777FEFFF7DBFEE0B2FFF759
:107E700072FEFFF7D6FEFFF79BFE3320FFF76BFE87
:107E8000FFF7CFFE0020FFF739FE0446FFF7ABFEF9
:107E9000204610BD10B50C46FFF7DFFF2070012013
:107EA00010BD70B50D460446FFF782FE3220FFF785
:107EB00052FEFFF7B6FEE0B2FFF74DFEFFF7B1FE50
:107EC0002846FFF748FEFFF7ACFEFFF78CFE0A20BE
:107ED00001F047FE70BD10B5FFF7E3FF012010BDB4
:107EE00010B50248FEF7F8FD10BD00008814002010
:107EF000FEB50446002572B60068394A831804D1DD
:107F00003849CD68032189040D4081680191C16819
:107F1000009141698669002B08D132484038836A54
:107F2000C7043B438362836ABB4383620846304392
:107F300048D02B482368C34205D12A48C36803228E
:107F400092049343C360002917D02068026901237B
:107F50001A43026120684161FEF7FCFC0746FEF708
:107F6000F9FC2168C01B0968090703D47D21C900F9
:107F70008842F4D9216808204860002E17D0206874
:107F8000016901221143016120688661FEF7E2FC6C
:107F90007D270646FF00FEF7DDFC2168801B09688F
:107FA000C90601D4B842F6D92168102048600C48AF
:107FB0002168C14206D10B48C16803229204914353
:107FC0002943C160206801694908490001612168AD
:107FD0000198886021680098C86062B6FEBD000004
:107FE0000084FFBF401002401CB5002116480091DC
:107FF000144A01910260C163120542608160072248
:108000008263012202610246C16020321170FF23A7
:108010005170C23343628162117301638161042232
:1080200041634261C161FEF795F8084800908013F2
:10803000019069460448FEF73DF800210248FDF72B
:10804000E3FF1CBD002401402C14002002000004AA
:1080500008B50848016B012211430163006B01213F
:108060001040009000220A20FEF762FE0A20FEF770
:1080700055FE08BD00100240F0B587B014216846D7
:10808000FDF795F84C48C26A04210A43C262C26AED
:108090000A400592C16A80273943C162C16A3940EA
:1080A0000591C16A01252943C162C16A2940059130
:1080B000C16A02263143C162C06A2A463040059037
:1080C00005201C210007FEF73EFC01223B493C48ED
:1080D000FEF739FC00223B493948FEF734FC912178
:1080E0000520002209020007FEF72DFC364801900A
:1080F000002405206946009502940007FEF75EFB08
:108100000320019005206946009602940007FEF7BF
:1081100055FB0C20009011200190032003900520B6
:10812000029469460007FEF749FB102000900520E5
:1081300069460396019502940007FEF73FFB112064
:10814000019002946946009503941D48FEF736FBA2
:108150001E4801906946009602951948FEF72EFBCD
:108160001B48009002946946019503941448FEF759
:1081700025FBE8026A4651C269461148FEF71EFB1C
:108180009120000200900520029469460195039415
:108190000007FEF713FB6946094800970295019412
:1081A000FEF70CFB002201210520FEF7C1FD052092
:1081B000FEF7B4FD07B0F0BD00100240010600005C
:1081C00000040050083000000000111000002110D1
:1081D0000836000010B50F4C0D482060FF20053018
:1081E00060600020A060E06020616061E0610121CA
:1081F000206249026062A161A0620720E06220461D
:10820000FFF7AEF92068016840221143016010BDFC
:1082100000300140B814002000B585B01421684634
:10822000FCF7C5FF0E480D490160E121490241609C
:1082300000218160C160016181610C22C1614261E4
:108240000162302141620121090381634900C16358
:10825000FFF7AAFA01F0C6F905B000BD00380140E9
:1082600010150020704700008307FF22DB0E9A40A4
:108270008907090E994000280BDA0007000F08381B
:10828000830808489B001818C36993430B43C361D4
:108290007047830804489B001B18186890430843E4
:1082A0001860704700ED00E000E400E0BFF34F8F7E
:1082B00004490348C860BFF34F8F00BFFDE70000CB
:1082C0000400FA0500ED00E0F0B585B00A2001F0E9
:1082D00025FF002001F03CFFFB4D0026AE70A87B7F
:1082E0000C2801D30B20A87301220520510200079E
:1082F000FEF729FBEE70F548AE74F54C007820715E
:108300000221F448FEF716FB002864D00020A9796A
:10831000EF4C49000843297D89000843E071A86AB1
:10832000E070401CA86268792146A0724200B43116
:108330000846A938FCF722FF06206072E249204671
:1083400013388A7F0275C97F417568790022400021
:1083500021460D3001F0CCFF6879002140000D303E
:1083600001F0D8FF022001F029FF0026E6712E74EB
:10837000AE7201202873EE72D748FEF78DFC688438
:108380000446EE706879FDF779F9D44AD44BFDF7CD
:108390006FF801F07BFB012300229B07FCF7B6FF7F
:1083A000FDF7B2F90006C00C001980B20121C90323
:1083B000A884884201D3401AA884CA4868632879EF
:1083C000401C2871C448FEF767FC2884C048C64C8E
:1083D0004E30029072E1012099E7BF48FEF75CFC45
:1083E0002884C24F0AE0BC48FEF756FC80B22884BD
:1083F000A98C884202D30919884206D300210F2094
:1084000001F00CFE3842E862EDD0E86A411C20D051
:108410002E4640047ED58122D20100210F2001F09A
:108420003CFF002001F094FE002001F046FE0021F8
:10843000102001F0F3FD4106A548490E00225030FE
:10844000019101F021FEA2485030417A0729C1D1A3
:1084500001E0FFF72BFF9E480222A5495530FCF7AB
:10846000B1FE0028B6D101F0A6FFF164B06401F0BE
:108470008FFF71653065F0786946401CF070944854
:108480004D3002790A70407948700888F18B884233
:108490007DD10298974F008A38808D488A494C30A8
:1084A000808A48838C48FEF7F7FB3084708B9249B2
:1084B000FF30C33080B2708388420CD949424018E3
:1084C000708338888C49401C80B20B3138808842D8
:1084D00001D30020388002987B4A81891186C089A7
:1084E0005086326B72637A4A5032D27C13071B0F6C
:1084F000032B00D0B3741209F274002333710123EB
:10850000B372714B002A9986D88615D00222784919
:108510006F4800E0C6E05530FCF754FE00280BD150
:1085200001206B493074C871019864311638C2B2A9
:1085300072747248FCF722FE0120F07264496248AE
:10854000042251314030FCF719FE6148736D16303A
:10855000326D01F005FF3F887D20C000718B7843AC
:108560004018B063049066480178F1736548019142
:10857000C088FDF768F800903846FDF764F8009968
:10858000FCF786FE7F21C905FCF729FE00E02DE0FF
:10859000FDF782F85A4980B208800199491E884245
:1085A00001D10120F072F7841620305EFDF752F8F9
:1085B00001910090308CFDF761F8534A534BFCF762
:1085C00057FF074603910498FDF744F83A46039B8A
:1085D000FCF740FF019B009AFCF798FEFDF770F84E
:1085E000F0634B48008800F0F3FB67E0FDF79EFB6B
:1085F0000746424803210C38C155029932488A89FE
:108600000286C98941863D49B8009C39326B0A50BF
:10861000E43940181A30736D326D01F0A1FE7079A3
:108620007F1C87424AD101F017FCFF23296D5B04B0
:10863000686D0022C918504100060C0A0443600806
:108640004000010E0002E965A8652148EB6C0A3084
:10865000AA6C01F085FE1E48EB6D1230AA6D01F088
:108660007FFE1B480821417268790022800018496A
:108670001C3001F03DFE6879002180001C3001F0C3
:1086800049FE204601F043FD012001F097FD000660
:10869000000E287241D100210F2001F0BFFC00061E
:1086A000F9D53AE03A4600210F2001F0F6FDF078C6
:1086B0007179884202D0002001F0FFFC298CA88C3F
:1086C000814227D289E6000048000020BC0000203B
:1086D000941100200004005088140020B81E85EB7F
:1086E00051B8CE3FA0860100983A000000D0272460
:1086F000D8000020E0000020E70300001413002051
:10870000D4000020200D0020F853E3A59B843E40B8
:10871000C400002000198142D4D86C4A00210F20E7
:1087200001F0BBFD6A4800240078002803D16948A5
:10873000008800F04DFB0027674938468F734A795F
:10874000039220E0624D295C00291AD0624B303D33
:108750009E7B761C9E73A300E9509C464300903D8F
:10876000ED5A66005A4B641CA83B9D538500183394
:10877000574E5D596346603EF550554B491EE4B275
:108780001954401CC0B29042DCD35348C17803292D
:1087900001D2817B817350490022887B4873401E3F
:1087A00035E000212FE04A4D8B00603DEC585E190A
:1087B00001967668B446644523DD00944C00483D3C
:1087C0002D5B9600AE46424D303DAD59404E029570
:1087D0006546603EF5503546483D6519AC466D88A6
:1087E000483E3553344678341E19394D7468303D4F
:1087F000EC50019C009B6360734665466B80029D54
:108800007560491CC9B28142CDDB521CD2B2824292
:10881000C7DB2F48603802682F48416B32398A42E3
:108820001ADA2B4930390968002915D0C179491C59
:10883000CAB2C271032A05D92549A8390A88C28358
:10884000012202700179032900D90770204C002110
:108850000378C03C039A08E0C771F3E74D00655BFD
:10886000002D00D10123491CC9B29142F6D30370F7
:10887000174B0021194A903B8C00491CC9B21A5170
:108880000C29F9D3007C002806D011490C31087856
:108890004B788A7802280ED00C4A002180320F20B3
:1088A00001F0FBFC01210520002249020007FEF730
:1088B0004AF805B0F0BD0A48C91CC018FCF75EFCB8
:1088C00001F0ACFE642001F045F9C2E500D0272498
:1088D00008130020C400002048000020FFFF010012
:1088E000200D002070470000F0B58DB0AF4801901A
:1088F0000020C0430A9000260A2001F00FFC00204F
:1089000001F026FC0020AA4C0546A070A94FAA48F9
:108910000B90A9480022C23885730146142001F04B
:10892000E7FC0021142001F0F5FC022001F046FCD8
:1089300000210F2001F072FB3842E062F8D0E06ABB
:108940000146401C18D048047ED58122D201002166
:108950000F2001F0A2FC0021102001F05FFB410676
:108960009548490E0022801C01F08EFB9248801C25
:10897000417A022902D0FAE0FFF798FC8E480222E1
:108980008E49C01DFCF71EFC0028F4D101F013FD38
:10899000E164A06401F0FCFC61652065002E23D138
:1089A0000B998748098A018083488149801E808A03
:1089B000488301268348FEF76FF92084608B824943
:1089C000FF30C33080B2608388420DD949424018DD
:1089D0007B49608308887C4A401C80B20B32088047
:1089E000904201D3002008800B98694682890A8052
:1089F000C089488070490422C91C0846A238FCF787
:108A0000BDFBFF22216D5204606D0023891858417F
:108A10000006090A01430846029101F078FB029919
:108A200048084000010E0002E165A0656248E36C61
:108A30009638A26C01F094FC5F48636D9238226D09
:108A400001F08EFC5C4800E093E08E38E36DA26D8F
:108A500001F086FC58490022A0393C2001F048FC76
:108A600000213C2001F056FC012001F0A7FB207200
:108A7000A0780121401CA0700520C9030007FDF764
:108A800069F94F487D2100880490C900059048434A
:108A9000618B4018A0630C904C480078E073039001
:108AA0004B48C088FCF7CFFD02900598FCF7CBFD42
:108AB0000299FCF7EDFB7F21C905FCF790FBFCF761
:108AC000EBFD81B2414801800398401E814201D1F3
:108AD0000120E0720498E0841620205EFCF7BAFDC5
:108AE00004910890208CFCF7C9FD3A4A3A4BFCF7F8
:108AF000BFFC069005910C98FCF7ACFD059B069A0F
:108B0000FCF7A8FC049B089AFCF700FCFCF7D8FDD6
:108B1000E0633248008800F05BF9009901988142D7
:108B20000DDA00290BD024490422C91C0AA8FCF73D
:108B300025FB012020700520607200980190207AAA
:108B4000002805D100210F2001F068FA0006F9D5B0
:108B5000802200210F2001F0A0FB00206D1CEDB24F
:108B60006070032D00D2D4E6002E08D01AE0012058
:108B7000F4E71B4A00210F2001F08FFBF7E7A08BE1
:108B80001849401E0004000CA08302D00A889042BD
:108B900001D90988A1831449A08B0988401E484344
:108BA0000E4908800A98E0830DB0F0BD3F420F00E7
:108BB0004800002000D02724E2110020D800002027
:108BC000E000002088140020E7030000D40000200B
:108BD000200D0020F853E3A59B843E40C4000020F4
:108BE00000902724C8000020C6000020F8B52D49B9
:108BF0002B48086001F0B2FC81202B4D800068807A
:108C0000E888002801D16420E880284801784329B9
:108C100001D943210170E98E0170254CE88F607104
:108C2000A88FA071A87AE070AE880521E661618105
:108C3000EF883846FCF75CFAA08101463046FCF725
:108C400057FA8800081886B27D20C000268170433C
:108C5000FCF714FD174A184BFCF772FCFCF754FDA7
:108C6000E0817D2066823946C000FCF741FA20820F
:108C7000E08201202083FDF771F8A082E2890F498C
:108C80000F48FEF70DF80FA0E16900F04DFDE988EF
:108C900010A000F049FD298913A000F045FDF8BDA2
:108CA0001D96000844000020200D00200000002038
:108CB000BC000020F853E3A59B843E40FF7F0000EA
:108CC00088140020B1EAC7A949443A202564202E1F
:108CD0000D0A0000CDA8D1B6BCE4B8F43A20256452
:108CE000206D732E0D0A0000B5A5B4CECDA8D1B667
:108CF000BBF9D5BECAFDC1BF3A202564B8F62E0D1A
:108D00000A00000070B586B014216846FCF74FFADF
:108D100001250F4EED03002229463046FDF713FED4
:108D20000120002401900294694600950394304686
:108D3000FDF744FD032001900294694600950394D9
:108D40003046FDF73BFD022000F004FF06B070BD89
:108D50000004005070470000F8B5044600206A4641
:108D60001080194D55222A70AA226A700322AA7017
:108D7000661DEE702A716971144A49008918AC7138
:108D80002246E81DFCF7FAF9002007E029186A4698
:108D90008978128889186A461180401CB042F5DB38
:108DA000611DA81CFCF746FE014668460180291992
:108DB0000078C87168464078087221460931024837
:108DC00000F08CFAF8BD0000C8130020200D002030
:108DD00010B514484178C38A8A00018B994201D3A7
:108DE000C91A01831049008BC988414388187D2125
:108DF000C90048430D490968401AFCF72BFC0C4A8E
:108E00000C4BFCF79DFBFCF75BFC0B49884201DD3A
:108E10004A428018002800DA401808490968486169
:108E200010BD0000BC000020200D002084000020A8
:108E3000F853E3A59B843E40FF7F00008814002088
:108E4000034A1168382389B299430143116070477E
:108E50000030014010B5FDF783FD10BD10B59AB08C
:108E600034216846FCF7A3F914210DA8FCF79FF9FB
:108E70001C2112A8FCF79BF91B4801680324E4029B
:108E8000A143C21489180160FDF75EFF174801690C
:108E9000A143016106200090FF20013002900120D3
:108EA0000390102004900220099040040B900001D0
:108EB00000240C900A946846FEF744F90F200D90A8
:108EC00003200E900F941094012111940DA8FEF729
:108ED00027F881201290032080041890149412A87F
:108EE000FDF76CFF1AB010BD00700040401002404A
:108EF00010480168821511430160C1680E4A114093
:108F0000C16001680D4A114001608168490849004B
:108F1000816001680122920491430160C168FD22D1
:108F200012049143C1600021016106490448886030
:108F300070470000001002400C40FF88F6FFF6FE6C
:108F40000050000800ED00E070B501F07BF81D4C0A
:108F50001D4D606402E001F075F86064A842FAD12A
:108F6000207801250526ED033607002804D00128C6
:108F70000FD0022823D120E0012229463046FDF7F8
:108F8000E2FCFFF7B1FC002229463046FDF7DBFC8E
:108F900015E0607A0122401E607229463046FDF7D6
:108FA000D2FCFCF7F7FE002229463046FDF7CBFC49
:108FB000607A002803D1207001E0FFF785F900F006
:108FC00033FF70BD480000203001CADE10B5818C2F
:108FD000C90707D001684A6801235B049A43836A82
:108FE0001A434A60818C890707D501684A680123C2
:108FF0001B049A43C36A1A434A60818C490707D508
:1090000001684A6801239B049A43036B1A434A6030
:10901000818C090707D501684A680123DB039A435D
:10902000436B1A434A60818CC90607D50268916870
:1090300001231B039943836B19439160818C89063B
:1090400007D501688A6801235B039A43C36B1A43FF
:109050008A60818C490612D503685A680121090586
:10906000046C8A4322435A60026C8A4207D1026828
:10907000516803235B059943436C19435160818C0C
:10908000090607D501684A680123DB04806C9A430E
:1090900002434A6010BD0000F8B500260446C667CA
:1090A000FDF758FC054620680068124F000709D5F7
:1090B00001212B46002249052046009700F054FA72
:1090C00000280DD12068006840070BD501212B46F0
:1090D000002289052046009700F046FA002801D0BA
:1090E0000320F8BD20206067A0676034267400204C
:1090F000F8BD0000FFFFFF01F8B5184CC826E07866
:10910000002829D16079002826D101206071144DF2
:10911000686B002700281ED0686BC821081A15E06C
:109120001048E168405C616988470F480A2100885F
:1091300048430E490880E068401CE060E068C828A9
:1091400000DBE760696BC820401A761EE168814247
:1091500001D0002EE4DC6771F8BD00003000002073
:1091600000000240580C0020CC000020D600002057
:1091700070B5224CE07800283FD1207900283CD1FE
:10918000012020711E4EF16900250906002933DAFD
:109190002156625791420AD1F06940062CD5A07938
:1091A000002829D0A5712089401C208124E0A179C4
:1091B000002903D1A0710A2000F0D3FC0020205622
:1091C000CC2148430F494218206912181279B26223
:1091D000401C00222061A256CC235A438958814268
:1091E0000ADC25612078401C207020780E2800D1F0
:1091F0002570A078401CA070257170BD3000002043
:10920000003801403001002010B5806A002201467C
:1092100040314A834A82FEF728FA10BD70B5846A4D
:10922000606FA56F2168896800260906002906DAA3
:10923000212804D152200653204600F047F8206828
:109240008068400606D5222D04D15A2006532046B8
:1092500000F02CF8E06F10210843E0672046FEF78D
:1092600004FA70BD10B501460968806A096889066C
:1092700014D400225A210A5201680A68FF230133DC
:109280009A430A6001688A68520852008A6001683D
:109290008A6840239A438A6020218167FEF780FB19
:1092A00010BD10B5806AFEF77CFB10BD01680A682E
:1092B000FF2321339A430A6001688A6852085200EA
:1092C0008A602021816700210166704701680A6871
:1092D000C0239A430A6020214167704770B5164C3D
:1092E000E278002A0CD12279002A09D10122E27009
:1092F0000025C82903DC0222A256002A01DCE57001
:1093000070BD0123E356CC2253430C4AD1500123B4
:10931000E356CC2673439B180A460146181DFBF7FB
:109320002DFF6078401C607060780E2800D1657059
:10933000A078401EA070E2E730000020300100203D
:10934000F8B504462669A268E769324366691020C9
:1093500000253E432368324378491E68784F3E40DB
:1093600016431E6023685A6803263603B243E66834
:1093700032435A602368A2698B4201D0266A324385
:109380009E680B273F02BE4316439E606D4E2368C6
:109390006D4AB3420CD1D2689207920F06D0012ACF
:1093A00038D0022A34D0032A20D11EE001201DE04B
:1093B000664EB3420AD1D2680C26324026D0042A27
:1093C00028D0082A24D00C2A10D10EE08B420DD1CF
:1093D000D66803229202164018D001229202B61AD1
:1093E00018D0B61A14D0964200D10820564A012649
:1093F000403A574FF6038B4236D100280CD0022852
:109400000DD0042812D008281FD11CE00020EDE761
:109410000220EBE70420E9E7FDF738FE08E01068DA
:10942000C00601D5384605E04A4803E0FDF74EFE88
:10943000002873D0626851005118814205D8110389
:10944000814202D303E03046F4E7012566E0010ED5
:1094500006025008002330185941FBF75FFE032134
:109460000902411A3C4A55E0E169B14232D1030098
:1094700000F081F909070A0D06250606062B0600ED
:10948000E3E7FDF703FE1CE0FDF710FE19E01068AE
:109490006168C00602D54808304A01E0304A4808F1
:1094A0008018FBF725FE80B201462E4A1039914202
:1094B000CBD8511C01400007400F08432CE0FDF7BA
:1094C00005FE616840004A08EAE761680122480831
:1094D0001204E5E7030000F04EF909070A0D06261D
:1094E0000606062C0600B0E7FDF7D0FD1DE0FDF7EF
:1094F000DDFD1AE010686168C00602D54808C01991
:1095000002E014484A081018FBF7F2FD80B2014649
:10951000144A1039914298D82168C860002020660A
:1095200060662846F8BDFDF7D1FD61684A088018DD
:10953000EAE7616848088019E6E700000048004053
:10954000F369FFEF00380140401002400044004042
:1095500000093D000024F400FFFC0F0000127A0017
:109560000048E801EFFF0000FFB581B017460E4646
:1095700004460A9D09E0681C07D0FDF7EBF9049941
:10958000401AA8420CD8002D0AD02068C169304684
:10959000884318D00020B842EDD0002005B0F0BDBF
:1095A00020680168FF22A132914301602068816830
:1095B00049084900816020206067A067002060346E
:1095C00020740320EAE70120E5E7000010B5044914
:1095D0001020096808620248FEF748F810BD000034
:1095E0001015002001490D208870704730000020C0
:1095F00010B507480A22018A51434183FEF728FD2E
:10960000FEF70AFEC82203490348FEF76DF910BDB4
:10961000BC000020580C002010150020F8B53D4C6F
:10962000002321783C4A1D46082910D0072945D03F
:1096300006294ED0052950D0042951D0032952D0F3
:10964000002954D0012956D0022958D059E0A178D8
:1096500000264A1F04E0304FBF5DFB189BB2761C0A
:109660009642F8DB667927799A195118E37862787F
:10967000C9188918C9194018C0071AD0012E14D06A
:10968000022E16D125482449C018FBF777FD00F0BB
:10969000C5FF642000F05EFABFF34F8F21492048D8
:1096A000C860BFF34F8F00BFFDE759081046FFF7B2
:1096B00053FB2570E570A570A571F8BDA1795054D4
:1096C000491CC8B2A071A178491F8842F5D1082071
:1096D00001E0607007202070F8BDE0700620FAE716
:1096E00060710520F7E7A070E5700420F3E75528C6
:1096F00007D10120EFE7AA2803D10220EBE70328D6
:1097000003D02570E570A570F8BD0320207020718E
:10971000F8BD0000B300002064130020200D0020DD
:109720000400FA0500ED00E00FB410B503A9044BE6
:10973000044A029800F002F910BC08BC04B01847B3
:1097400079A30008F00000202021020C01D0102194
:109750001046020A01D010460839020901D010460D
:10976000091F820801D01046891E420801D0881EB8
:109770007047081A704730B47446641E2578641C1C
:10978000AB4200D21D46635D5B00E31830BC184756
:1097900002E008C8121F08C1002AFAD170477047BA
:1097A000002001E001C1121F002AFBD1704708B55B
:1097B0000021684601706B46012202212C2000F036
:1097C0007BFD0221684601706B4601222C2000F0CF
:1097D00073FD08BD38B504466D20694608706B46B8
:1097E000012207492E2000F067FD0649002C01D018
:1097F000054A00E0054A2E2000F044FD38BD000077
:109800000608000006180000070600000716000002
:1098100038B504466B4602220021362000F018FCC1
:10982000B3212300FFF7A7FF0E0F08153A3A3A3A83
:109830001C273A3A2F34483A002168460170407894
:109840004108490014E06946087880088000401CFF
:1098500004E06946087880088000801C08701DE0DC
:10986000684602780A4048320270417880200143FD
:109870006846417012E0684602780A4002704078FB
:109880004106490EF4E7694648780221084303E09F
:1098900069464878FD210840694648706B460122B8
:1098A0000021362000F008FD012200AB11463620D1
:1098B000013300F001FD38BD69460878CF2108402A
:1098C00069462030CAE708B5032168464170012186
:1098D00001706B4602220021362000F0EDFC0122CF
:1098E000D20306212D2000F0CDFC012000F032F93A
:1098F0000120FFF78DFF08BD08B5020A69464A70CE
:1099000008706B46022204212D2000F0D5FC0320B4
:10991000694608706B46012206212D2000F0CCFC20
:109920000020694608706B46012206212D2000F0B8
:10993000C3FC0A212D2000F071FB08BDFFB58DB0DE
:109940000446002506E025280AD0109A0F99904772
:10995000641C6D1C20780028F5D1284611B0F0BD9C
:1099600000270121484A009700E00743641C237840
:109970000846203B98401042F7D120782E2817D176
:10998000042007436078641C2A280CD10E98641CBC
:1099900002C800910E900BE000990A225143303921
:1099A0004018641C00902078014630390929F3D909
:1099B00020780028D1D0642808D0692806D07528DE
:1099C0001ED0109A0F9990476D1C5BE00A200E99EB
:1099D000019001C90E91002802DA40422D2102E0D7
:1099E000390504D52B216A461172012103E0F907DC
:1099F00004D02021F7E70BAE0B910DE00021FAE730
:109A00000A200E99019001C90E91F7E70199FBF721
:109A10006FFB3031761E31700028F7D103A8801B10
:109A200020300190780701D5009801E001200090D6
:109A30000199884201DD401A00E0002000270090D3
:109A400006E002A8109AC05D0F9990476D1C7F1C1C
:109A50000B988742F5DB04E0109A30200F9990476D
:109A60006D1C0099481E00900029F5DC05E0307857
:109A7000109A761C0F9990476D1C0199481E019011
:109A80000029F4DC641C65E709280100F8B54A00E8
:109A90002B4B520DD6182B4A0C460546142E2BDAAA
:109AA000002E12DA284BFBF731FC00221346FBF79D
:109AB00057FF40D2002C03DA0124E40700253AE0E6
:109AC0002046284337D0214C14E0214F0B46F74065
:109AD0003B402B4331D01C4BFBF718FC00221346B4
:109AE000FBF73EFF27D2002C03DD01200005F040EC
:109AF0000419BC4300251EE0332E1EDC334600272C
:109B0000143BFF43DF40384217D00F4BFBF7A8FC54
:109B100000221346FBF724FF0DD2002C0ADD142E81
:109B20000CD03420811B012088404019A84200D26B
:109B3000641C0546BD4321462846F8BD641CF9E770
:109B400001FCFFFF9C7500883CE4377E0000F03F7D
:109B5000FFFF0F007D2110B5C900484300F001F858
:109B600010BD002140E000BF00BF00BF00BF00BF2C
:109B700000BF00BF00BF00BF00BF00BF00BF00BFED
:109B800000BF00BF00BF00BF00BF00BF00BF00BFDD
:109B900000BF00BF00BF00BF00BF00BF00BF00BFCD
:109BA00000BF00BF00BF00BF00BF00BF00BF00BFBD
:109BB00000BF00BF00BF00BF00BF00BF00BF00BFAD
:109BC00000BF00BF00BF00BF00BF00BF00BF00BF9D
:109BD00000BF00BF00BF00BF00BF00BF00BF00BF8D
:109BE00000BF00BF00BF491C8142BCD370470000CA
:109BF000FEB5044600200190009060797349400052
:109C00000E5A61782578491E7148CFB20163042D40
:109C100077D0072D75D000210291217801736C490E
:109C2000E379012292058969002B6CD0914381610F
:109C30006748217A4173217A82698907890B0A432F
:109C400082610021042000F028FB324661492E2069
:109C500000F018FB3846FFF7BDFD5F4E0522705D32
:109C6000810040185D49431807212B2000F024FB98
:109C70005B49029801220B180B21282000F01CFBE5
:109C8000705D584980000A580C21282000F005FB1F
:109C9000E079554980004018A1794900425A0221D3
:109CA000272000F0EFFA51487E00825B0421272034
:109CB00000F0E8FAE079002829D0A07804282CD018
:109CC00028206946087220220621272000F0DAFAAF
:109CD00002AB01222621272000F0EEFA4449380188
:109CE0004018E178890042580821272000F0D5FA71
:109CF000A17A601C627A0902114313D016E000E0D9
:109D000001E0012188E71143F608816190E76422B0
:109D10000621272000F0B6FAE0E710206946087215
:109D20000246D1E733490172090A4172417A007A49
:109D30000A0202432021272000F0A4FA2E4F0C2112
:109D400023203A6800F0A9FAF01982880421232020
:109D500000F098FAA07900280BD0E0792749012279
:109D600043180021212000F0A7FA032001900120D0
:109D700000902A07120F100102436078002180072B
:109D8000000B02430198000502430098400402437F
:109D90002079C006400902436079C00602431F20B3
:109DA00000F07BFAA0786178012308430204084898
:109DB000DB030261E179490319430A43026100218F
:109DC000082000F06AFA0020FEBD0000E8A60008A6
:109DD000F40000200428000090A6000801000020E4
:109DE0001F00002098A60008B8A60008C4A6000816
:109DF000C8A6000841100000B0A6000821000020FD
:109E000038B50C4607498A8B002102432C2000F00C
:109E100039FA684604706B46012206212C2000F0B6
:109E20004BFA38BDF400002010B5FFF7C0FC10BDA0
:109E300010B504460421362000F0F0F80121C902D3
:109E4000002C01D0084300E088430246042136205C
:109E500000F023FA10BD000038B5402069460870B4
:109E600000210E2000F0DAF80446002211460E20F0
:109E700000F013FA6B46012200210D2000F01CFABD
:109E8000074A00210F2000F008FA00F0E1F922460D
:109E900000210E2000F001FA02480021017338BDB4
:109EA000F8FF2724140100207CB5054604206946EC
:109EB00008704B4C002060752146203120634871AA
:109EC0000873A0836063A06300F0BCF8454E206077
:109ED00002E000F0B7F82060B042FAD10020FFF7AE
:109EE00097FC41480078242801D9243806E006214F
:109EF000FBF7FEF80622101A40010843020601048F
:109F00000A4301020A43024300211E2000F0C5F962
:109F10006B4601220021242000F0CEF91E20FFF71D
:109F2000EBFC86B2300AA0730420FFF7E5FC0006C4
:109F3000000E0DD002206946087101AB01221221EA
:109F40002D2000F0B9F9A08B012109030843A0835B
:109F500000F078F820600620FFF7CEFC6060072054
:109F6000FFF7CAFCA060F006C00E207501D11020DA
:109F70002075C0B200F0DCF9E80707D0FFF7A3FCBA
:109F8000A08B0121C9020843A0830AE005213620E5
:109F900000F02EF81549084002460521362000F051
:109FA00071F90120FFF734FC0021042000F036F89D
:109FB000A0610021262000F031F815218903084313
:109FC00002460021262000F068F9002226213620D2
:109FD00000F058F900F036F8206000207CBD000049
:109FE000F40000203001CADE00000020FFFD000068
:109FF00038B5094C89B280B26B46022200F028F8CD
:10A00000002806D1684640780102684600780818A2
:10A0100084B2204638BD0000FFFF000038B50024A0
:10A02000E44389B280B26B46042200F011F80028A4
:10A0300006D103216846435C2202D418491EFAD592
:10A04000204638BD10B500210846FFF7E7FF10BDD8
:10A0500038B5002909D0402420436C462070C8B28E
:10A060007F2906D8607002200AE069460870012046
:10A0700006E0802420436C466070C809A07003206D
:10A08000694600F0A5FA38BD10B5144603460A46E5
:10A0900021461120FFF7DCFF10BD10B50346052255
:10A0A00000211520FFF7D4FF10BD10B5034605228F
:10A0B00000211720FFF7CCFF10BD38B50546002062
:10A0C0006946087000F0C4F8FF2401342246002DD0
:10A0D00001D00322120200210D2000F0D3F8002D40
:10A0E00013D06B46012203210F20FFF7B1FF684612
:10A0F0000078000709D5FFF7AFFE224600210D20AA
:10A1000000F0C0F80020C04338BD002038BD10B5B5
:10A11000024601210A2000F0C0F810BD10B5044627
:10A1200000211A20FFF77AFF000D22030005120B11
:10A13000024300211A2000F0B0F810BD10B502460D
:10A1400002492E2000F09EF810BD00000418000007
:10A15000F8B505466B46012203210420FFF778FF7E
:10A160000126114C3607002D0DD02A4600210C2067
:10A1700000F088F86946087810210843694608709D
:10A18000A069304307E069460878EF210840694636
:10A190000870A069B0430B46A0610122032104208E
:10A1A00000F08AF8F8BD0000F400002010B5024667
:10A1B0000021182000F066F810BD0000F8B5074631
:10A1C000002568460570B807204C2E4600280ADA9C
:10A1D0008020694608706B46012200210D2000F0A6
:10A1E0006BF801202073F8076946087821D0062112
:10A1F0000843694608706B46012200210D2000F0DB
:10A200005BF803210F20FFF7F3FE8121C90008420C
:10A2100019D04020694608706B46012200210D20AC
:10A2200000F04AF80020FFF703FE00252673ED43F7
:10A2300009E002210843694608706B4601220021AB
:10A240000D2000F039F82846F8BD00001401002068
:10A250001CB56B46012203210F20FFF7F9FE68466B
:10A2600000784022C1091040C9014000814208D055
:10A27000012069460871024601AB03210D2000F060
:10A280001BF81CBD08B56B461A70120A5A7089B2C9
:10A2900080B2022200F010F808BD38B500236C46E9
:10A2A000E254120A5B1C042BFADB89B280B223460B
:10A2B000042200F001F838BD38B58024002909D007
:10A2C000C02528436D462870C8B27F2907D868701A
:10A2D000022009E0204369460870012004E0204381
:10A2E0006870C809A8700320694600F0ADF938BD50
:10A2F00010B51446012312189B029A4202D900207D
:10A30000C04310BD0B46821E21460920FFF7D4FF33
:10A31000002010BD10B5054A8905126901430A43A2
:10A3200000210820FFF7B9FF002010BDF400002035
:10A3300038B504466B4601220E212B20FFF788FE1C
:10A3400068460078E10640094001C90E01436846AD
:10A3500001706B4601220E212B20FFF7ADFF38BDA7
:10A3600010B5002142541C06120A22431B0A491C44
:10A370000429F7DB10BD000013B501231A46694616
:10A380000248FDF70FFB00981CBD000010150020CF
:10A390007CB5002425466846FFF77FFE0420694609
:10A3A000220E2D02154322020C5C1443401EF7D5E9
:10A3B000204629467CBD7CB5002425466846FFF72B
:10A3C00074FE04206946220E2D02154322020C5C05
:10A3D0001443401EF7D5204629467CBDFCF7C8FA39
:10A3E000FEF73CFDFDF748FE37493848002522C0FE
:10A3F00005608561C56136490562C1600838FCF7B2
:10A40000D1FBFDF725FEFDF707FFFDF7E3FEFDF7A6
:10A41000EBFD052601223607D1033046FCF793FAFF
:10A42000FEF7E4FBFDF7E4FCFBF764FBFBF732FB14
:10A430000721B015FFF7E4FC264C0A21208A0122EF
:10A4400048436083170339463046FCF77CFA1F48BF
:10A45000C82221498830FDF747FA204E207900288C
:10A460002FD0FEF7FBFC2571FBF75AFD20700F285B
:10A4700009D9012239463046FCF765FAFEF764FD3A
:10A480000022394609E0012251033046FCF75BFA0D
:10A49000FEF75AFD0022012149033046FCF753FA2A
:10A4A000FDF7EAFB608B002801D0401E60830C485A
:10A4B000618B00780843D1D101210846FCF764FC88
:10A4C000CCE7FDF7D9FBC9E7007C004088140020E9
:10A4D000FFFF0000BC000020580C002000040050CA
:10A4E0003600002010B586B01748FCF7E0FA1421BA
:10A4F0006846FAF75CFE15480090032001900020A2
:10A500000290052069460007FCF758F96946104893
:10A51000FCF754F969460F48FCF750F90121084649
:10A52000FCF732FCFF2401342046FCF705FC0A4905
:10A5300008680422104308602046FCF70DFCFCF775
:10A5400013FC06B010BD000088140020FFFF0000BF
:10A5500000040050000800500070004010B50122B7
:10A56000920218491848FBF73BFB16481749028826
:10A570008A4225D0018004218180FF21F531C180EC
:10A580000A21018100211E224181D24382810122C0
:10A59000C2810184018241828182C18201838183DF
:10A5A0004323C38602230387782343878287C28796
:10A5B00002464032118451849184C18300F02EF808
:10A5C00010BD0000200D002000FC0008AA5500006E
:10A5D000F0B58C4600251026052109078E620E4C29
:10A5E00008E067467F5DE760A768FF07FCD0E76883
:10A5F0001F706D1C8542F4DB0020074606E0E76013
:10A60000A568ED07FCD0E5681D54401C9042F6D3C8
:10A610008E610020F0BD00000030014070B572B6C0
:10A620000124074DA40221462846FBF7BFFA002863
:10A6300004D0224603492846FBF75CFB62B670BD96
:10A6400000FC0008200D0020F0B50025102605278D
:10A650009C463F070B46BE620C4C06E0595DE1602C
:10A66000A168C907FCD0E1686D1C8542F6DB0020BB
:10A6700007E06146095CE160A168C907FCD0E168B8
:10A68000401C9042F5D3BE610020F0BD0030014077
:10A690000000010203040005405C0000A05C04000F
:10A6A000C06C0800805C0400E03F1E00E07D1E00DE
:10A6B00007A9022570889B880A0016000100060081
:10A6C0000100020087008D002D001A3152001A335C
:10A6D0009A001A351D011A376B003B31BE003B331F
:10A6E0005E013B3596023B37000099599959EB5171
:10A6F0008F421E45142E0080EB51F5283333E13A8A
:10A70000703DE13AC235852BC2353333C235C2358F
:10A71000AE47E13A5138A330513800000000000044
:10A7200000000102030406070809030406080C10D0
:10A730001820300000000001020304005CA700089C
:10A7400000000020F40000009097000850A80008C6
:10A75000F400002044190000A0970008000704003E
:10A76000091E08054008260910400856080540083B
:10A77000261D040008BE1D040008BED8BC401008F9
:10A78000010000000000C8420000000000000000BE
:10A7900000000000000000000000000000000000B9
:10A7A00000000000000000000000000000000000A9
:10A7B000000000000000000000005C12000000002B
:10A7C0000000000000000000000000000000000089
:10A7D0000000000000000000000000000000000079
:10A7E0000000000000000000000000000000000069
:10A7F0000000000000000000000000000000000059
:10A8000000000000020204000909010200810000AA
:10A810000000000001000000000400000000000033
:10A820000000000000000000000000000000000028
:10A830000000000000000000000000000000000018
:10A8400000000000000000000000200000000000E8
:04000005080050C1DE
:00000001FF
